:020000040000FA
:10000000A8260020F90200000103000003030000FD
:1000100005030000070300000903000000000000C2
:100020000000000000000000000000000B030000C2
:100030000D030000000000000F030000110300008A
:100040001303000013030000150700001303000052
:10005000130300001303000013030000A1030000BA
:10006000C506000013030000130300001303000083
:100070001303000013030000130300001303000028
:100080001303000013030000130300001303000018
:100090001303000013030000130300001303000008
:1000A00013030000130300001303000013030000F8
:1000B0001303000013030000000000000000000014
:1000C00013030000130300001303000013030000D8
:1000D00013030000130300001303000013030000C8
:1000E00013030000130300001303000000000000CE
:1000F00000000000130300000000000013030000D4
:1001000000000000000000000000000000000000EF
:1001100000000000000000000000000000000000DF
:1001200000000000000000000000000000000000CF
:1001300000000000000000000000000000000000BF
:1001400000000000000000000000000000000000AF
:10015000000000000000000000000000000000009F
:10016000000000000000000000000000000000008F
:10017000000000000000000000000000000000007F
:10018000000000000000000000000000000000006F
:10019000000000000000000000000000000000005F
:1001A000000000000000000000000000000000004F
:1001B000000000000000000000000000000000003F
:1001C000000000000000000000000000000000002F
:1001D000000000000000000000000000000000001F
:1001E000000000000000000000000000000000000F
:1001F00000000000000000000000000000000000FF
:10020000DFF80CD000F0BAF800480047F10B00000E
:10021000A826002030B4044654E8000F0D4644E8F8
:100220000053002BF8D1156030BC704730B4044641
:1002300054E8000F40EA010544E80053002BF7D1D1
:10024000156030BC704730B4044654E8000F00EA33
:10025000010544E80053002BF7D1156030BC70470E
:1002600030B4044654E8000F80EA010544E8005326
:10027000002BF7D1156030BC704730B4044654E809
:10028000000F00EB010544E80053002BF7D1156087
:1002900030BC704730B4044654E8000FA0EB0105B1
:1002A00044E80053002BF7D1156030BC704770B4A0
:1002B00004464FF0000054E8006F0D68AE4207BFDF
:1002C00044E80023012044E800630E60002B1CBFBB
:1002D0000020F0E770BC704730B4044654E8000FCB
:1002E00088422CBF451A054644E80053002BF5D13F
:1002F000156030BC7047000006488047064800473C
:10030000FEE7FEE7FEE7FEE7FEE7FEE7FEE7FEE7C5
:10031000FEE7FEE7E9040000010200000048704724
:10032000942E000040EA01039B0703D009E008C9AE
:10033000121F08C0042AFAD203E011F8013B00F8AA
:10034000013B521EF9D27047D2B201E000F8012BF6
:10035000491EFBD270470022F6E710B513460A4645
:1003600004461946FFF7F0FF204610BD421C10F866
:10037000011B0029FBD1801A70470000064C074D75
:1003800006E0E06840F0010394E807009847103465
:10039000AC42F6D3FFF738FF0833000028330000E3
:1003A0002DE9FE434FF48278404601F0B1FA4C4FFC
:1003B00000254C4C012600B3404601F0B1FA94F8F8
:1003C0002E0010B194F82F10D1B18DF80050616853
:1003D00001912189ADF80810E26832B1218B618367
:1003E00062602181E56010B102E0257400E03E60AA
:1003F00021686846884784F82F5094F82E0060B32F
:100400004FF48077384601F083FA30B3384601F074
:1004100087FA628B94F82D108A420AD9A2EB010068
:1004200080B260832289A2EB0000626802EB400088
:1004300005E007D1E06828B184F82F60658301F0FA
:1004400055FA04E08A4202D184F82F606583404661
:1004500001F066FA2248001D06604FF4887738469E
:1004600001F056FA48B1384601F05AFA25740220D4
:100470008DF800002168684688474FF48A7738462F
:1004800001F046FA28B1384601F04AFA2574BDE871
:10049000FE834FF000484FF48C7967691DE000BF80
:1004A000B7FA87F028FA00F109EB80058F43284658
:1004B00001F02EFA88B1284601F032FAA5F58C75C4
:1004C000E8088DF8040045F38000401C8DF80060BA
:1004D0008DF80500216868468847002FE0D1D6E7EF
:1004E00000700040E800002030B54FF0805000223E
:1004F0008300D0F83011C3F80C21C3F81021624BEF
:100500001A60624B1B68624C2360604B1B1D1B68AA
:10051000241D23605D4B08331B68241D23605B4B47
:100520000C331B68241D2360584B10331B68241D9B
:100530002360564B14331B68241D2360534B183320
:100540001B68534C20342360504B1C331B68241D04
:1005500023604E4B20331B68241D23604B4B2433F8
:100560001B68241D2360494B28331B68241D23600E
:10057000464B2C331B68241D2360444B30331B68CF
:10058000434C40342360414B34331B68241D2360AB
:100590003E4B38331B68241D23603C4B3C331B68A7
:1005A000241D2360394B40331B68241D2360012424
:1005B000082902D1D0F8343113B1082904D006E05B
:1005C000354B3449196005E0D0F8343113B10829AE
:1005D00004D006E0314BFB21196005E0D0F834313E
:1005E00013B1082908D00EE090F858322C48016861
:1005F00063F30301016002E0D0F834311BB92949EB
:100600004FF40070086028480168C90702D06FF0F5
:10061000010101602548016841F470010160BFF3E8
:100620004F8FBFF36F8F4FF01021D1F800020028D9
:1006300003DBD1F80402002822DA1D4B1C601D48A0
:100640000468002CFCD01224C1F800420568002D7B
:10065000FCD0C1F8044201680029FCD01A6001688E
:100660000029FCD0BFF34F8F10487C380168124A34
:1006700001F4E06111430160BFF34F8F00BFFDE75C
:100680000F490E48086030BD3805004004040010D2
:1006900020C50040488103008C56004018F50040FA
:1006A000E40E0040409602400004004088ED00E067
:1006B00004E5014000E401400400FA050090D00385
:1006C000B00000202DE9F047104E042700244FF41D
:1006D000A0784FF4803900BF08EB840509FA04F0D4
:1006E000715961B1D6F80413014208D02946304649
:1006F00001F05EF90648D0E9002128469047641CC5
:10070000E4B2BC42E8D3BDE8F087000000800040BE
:100710001801002001480068004700002800002060
:1007200002E008C8121F08C1002AFAD170477047BA
:10073000002001E001C1121F002AFBD17047000018
:1007400072B600F0CBFF00BF00F006FE0028FBD120
:10075000104C0121208801EB00400FA100F008FFA0
:1007600010480068C00700D000BE2088022101EBBD
:1007700000400DA100F0FCFEBFF34F8F0948E438A4
:1007800001680D4A01F4E06111430160BFF34F8F2E
:1007900000BFFDE7D0000020466174616C206572E7
:1007A000726F7200F0ED00E053797374656D207222
:1007B00065736574000000000400FA050EB50021A1
:1007C0000091CDE901106A4644F20100FFF7B8FF3D
:1007D0000EBD00F003B800F009B8000072B6024880
:1007E0000168491C01607047300000200349086817
:1007F000401E086000D162B6704700003000002043
:1008000070B5054608680C46411C04D000F0B8FCE1
:10081000206800F085FC6068411C02D0002100F0D7
:100820006DFC2968A069C1F82405607D227D2968D6
:100830001043C1F86C05D4E900122868C0F81425EB
:10084000C0F80C15207D012814D1A068411C02D0ED
:10085000002100F053FCE068411C04D000F090FC43
:10086000E06800F05DFCD4E902122868C0F80825B1
:10087000C0F8101570BD70B5054608680C46411CDF
:1008800004D000F087FC206800F054FC6068411C34
:1008900002D0002100F03BFC2968A069C1F82405C2
:1008A000607D217D2A680843C2F86C05D4E90012F6
:1008B0002868C0F80C15C0F81425207D012814D133
:1008C000A068411C02D0002100F021FCE068411C1E
:1008D00004D000F05FFCE06800F02CFCD4E90212C8
:1008E0002868C0F80825C0F8101570BD2DE9F0473C
:1008F0000546861C90460F464FF001090020FFF781
:1009000068FF1B4C20683860D4E90001401AA168D8
:1009100004F21C47081A0EE00121384600F0FCF9E9
:1009200000F018F90146384600F0F6F9D4E9000164
:10093000401AA168081A401C8642EDD8B8F1000F91
:1009400003D0052065F3891002E0062065F39F506F
:10095000A2682168114004EB8101C860206830441E
:1009600020600020FFF737FF4846BDE8F087000011
:100970008002002030B482680468531C8360A15454
:10098000D0E901128A4202D330BC00F07ABA30BCFE
:1009900070470000034803C8814201D1012070471D
:1009A000002070478002002010B50021024800F0AE
:1009B000BEF980F3100010BD9C0600202DE9FC5FFD
:1009C0000E008346DDE90C47C6F1000098469246CA
:1009D000814600D40846012503E000BF90FBFAF0F1
:1009E0006D1C5045FADAA84500D9454624B1002EC1
:1009F00001DB780700D5641EB80702D5B8F1000FF7
:100A00000AD0F80708D13CB1A54205D220215846AA
:100A1000641EFFF7AFFFF6E7002E02DA4E462D21E7
:100A200002E0780703D52B215846FFF7A3FF07F014
:100A3000030002280BD1B8F1000F08D13CB1A54248
:100A400005D230215846641EFFF794FFF6E7CDE942
:100A50000047434652463146584602F00DF8BDE87D
:100A6000FC9F000070B50D46044600684FF4887185
:100A700000F0BAFF4FF49071206800F0B5FF4FF41A
:100A80009271206800F0B0FF4FF4A271206800F06E
:100A9000ABFF20681249C0F8041320686907000BF7
:100AA00040B2090E002806DA00F00F0000F1E02045
:100AB00080F8141D03E000F1E02080F800142068A5
:100AC0000121000B40B200F01F029140400980005C
:100AD00000F1E020C0F88012C0F8001170BD0000E5
:100AE00010030200024600201268930702D0530749
:100AF00002D47047500714D502F00300012802D039
:100B000002280CD105E0C2F383100B68801C184446
:100B100004E00223086803EB9252104408600120AD
:100B20007047086800EB9253C2F38910401CEEE74F
:100B30000121814003484068014201D001207047F3
:100B4000002070472000002001218140080300D0D0
:100B5000012070472DE9FF410026234800F0D9F815
:100B60002148001F074600F0D4F8204C6068009030
:100B7000A56800E000986946284004EB80000C302E
:100B8000FFF7B0FF0028F5D101AA009901EA05039B
:100B900004EB8303491CDB6842F82030401C0091C1
:100BA0000228F2D3019800F0030001280BD002289C
:100BB00010D10198032101EB90500099BDF80A6013
:100BC00001EB900005E00198BDF80A60C0F38310C6
:100BD00008440090384600F099F808B10098606029
:100BE00004B03046BDE8F081980600208002002065
:100BF0004FF40041002000F02DFD08B1FFF7DEFDAD
:100C000000F09CFB00F044FE08B1FFF7D7FD01F0B7
:100C1000C1FC01F0F9FC01F0E9FC0848032100885F
:100C200001EB004006A100F0A3FC00BF00F044FE71
:100C300000F092FB0028FBD1F8E70000D000002074
:100C400053414144432048414C2073696D706C65A9
:100C5000206578616D706C65207374617274656471
:100C60002E0000002DE9F047C7880446181D1646DF
:100C70008946B0FBF7F1B0FBF7F207FB12009A19B7
:100C80003A44D21CB2FBF7F2DDF820A001E0246860
:100C9000491E0029FBD13D1A8846B54216D818E0F6
:100CA000BAF1000F05D0211809EB08002A46091DEA
:100CB00004E0204409EB08012A46001DFFF732FB3F
:100CC00000202468761BA844B74201D9354600E0CD
:100CD0003D46002EE4D1BDE8F087000030B5024665
:100CE00059B100F0E3FC0021074C09E004EB81035B
:100CF00015685B88AB4202D11160002030BD491CF1
:100D00008142F3D3052030BDB4000020002100F063
:100D100009B8012100F010B808B56A46FFF7ADFA2E
:100D2000009808BD08B56A46FFF78DFA08BD08B5FA
:100D30006A46FFF76FFA08BD08B56A46FFF776FA0C
:100D4000009808BD08B56A46FFF7A4FA009808BDE8
:100D500070B5044600252846FFF73BFD2168626810
:100D6000086890420ED9401E08600178A38AE268A4
:100D700001FB0325227A2168101AC0B20A79824247
:100D800000D208710020FFF726FD284670BD70B51F
:100D900005460C460020FFF71CFDE868A98A201ACA
:100DA000B0FBF1F12A681068431C13600170BDE8C4
:100DB00070400020FFF70FBD10B530B1017A4268D6
:100DC0000368891AC9B21A6006E00E2010BD0368D4
:100DD0001A68541C1C601170491EC9B2F7D2006811
:100DE00000210171084610BD0448017809B1852031
:100DF00070470121017000207047000008000020AA
:100E0000F0B505460478154889B0164640F8242008
:100E1000124A08690832A2F10C0742F82400487F00
:100E2000385520226846FFF77DFA04942878385C0C
:100E300048B10EB10A4A00E000226946281D01F0BF
:100E4000DFF909B0F0BD0EB1064A00E000226946A4
:100E500005F10C0001F0A6F8F3E7000010000020F7
:100E600055290000A12700000FB408B503990029F7
:100E700004D004AA00926A4600F00FF801B05DF8B1
:100E800014FB10B582680446002A05D0D4E9040397
:100E9000216898470020A06010BD2DE9FC479146CD
:100EA0000C00804676D014F8011B39B125290ED0EC
:100EB0004046FFF75FFD20780028F4D198F80C0039
:100EC000002867D04046BDE8FC47FFF7DABF0020A6
:100ED000012221782B291BD02D2902D0302908D1BD
:100EE00002E040F0010001E040F00200641C002A32
:100EF000EFD100252A290ED02178A1F130020A2A4B
:100F000011D205EB850201EB4205641C303DF1E78F
:100F100040F00400EAE7D9F800100B1DC9F80030D2
:100F20000968641C0D44217800232E290BD114F884
:100F3000011FA1F130020A2A05D203EB830201EB63
:100F40004203303BF3E76C290DD068290BD06929A7
:100F500021D00BDC252918D0582931D063290ED097
:100F6000642915D117E014F8011FECE7702969D046
:100F7000732932D075291BD0782909D120E0D9F8FE
:100F80000000011DC9F8001001784046FFF7F2FC8F
:100F9000641C90E76CE0D9F800100A1DC9F8002025
:100FA0000968CDE900500A224046FFF707FDEFE748
:100FB000D9F800100A1DC9F8002009680A2206E0C5
:100FC000D9F800100A1DC9F8002009681022CDE9DF
:100FD0000050404601F050FDDAE7D9F80010002734
:100FE0000A1DC9F800200E68C00705D112E040466E
:100FF000761C7F1CFFF7BEFC31780029F7D104E096
:10100000202140466D1EFFF7B5FCBD42C0D9002D22
:10101000F6D1BDE74EB13046FFF7A8F9074604E028
:10102000202140466D1EFFF7A5FCBD4206D9002DCC
:10103000F6D103E04046761CFFF79CFC317800298E
:10104000F8D1A5E7D9F80000011DC9F8001005681E
:1010500030214046FFF78EFC78214046FFF78AFC9E
:1010600008200021CDE90001034610222946B0E7FF
:10107000BDE8FC872DE9FF411C46DDE90A781546ED
:101080000E46684600F060F846EA450141EA8401F0
:1010900041EA072242EA0841009A00EB8200C0F8C8
:1010A0000017BDE8FF812DE9FF411C46DDE90A7804
:1010B00015460E46684600F055F846EA450141EAF5
:1010C000840141EA072242EA0841009A00EB8200CB
:1010D000C0F80017BDE8FF811CB5002100910B4648
:1010E00001220191FFF7C6FF1CBD1CB50021009134
:1010F0000B4601220191FFF7D6FF1CBD1CB5002253
:101100000B46009211460192FFF7B4FF1CBD1CB5BF
:1011100000220B46009211460192FFF7C4FF1CBD4E
:101120001CB5002100910B46012201911146FFF7E9
:10113000A1FF1CBD1CB5002100910B4601220191AD
:101140001146FFF7B0FF1CBD0168202902D24FF005
:10115000A040704701F01F01016001487047000086
:10116000000300500168202902D24FF0A0407047D0
:1011700001F01F01016001487047000000030050AA
:1011800001B56846FFF7E0FF009A01219140C0F8E1
:10119000081508BD01B56846FFF7E4FF009A012174
:1011A0009140C0F8081508BD30B5124B014600202B
:1011B000D3F81044224609E0157A854205D1401C37
:1011C0000A28F7DB4FF0FF3030BD5268002AF3D118
:1011D000421CF9D00872D3F810242AB152684A6030
:1011E000D3F81024516030BD0022C3F810144A60B7
:1011F00030BD000080020020F0B595B01C461546B9
:101200000F4608461A9E00F021FB182109A8FFF797
:10121000A2F80E96CDE909540023082203A9384606
:1012200000F029FB05980690BDF81000ADF81C00F1
:10123000BDF81200ADF81E0000208DF821000398C3
:10124000082600F00300012802D0022818D032E05E
:1012500003983346850AC0F3C2008DF82000039836
:101260000FA9C0F38314A200384600F004FB09A8BC
:10127000009006AB22460FA9284600F043FA1AE078
:101280000398840DC0F3C2008DF82000082C01D211
:10129000254600E0082533462A460FA9384600F0C7
:1012A000EAFA2E44641B09AB06AA29460FA800F0EF
:1012B0007BF9002CEAD1384600F0CEFA15B0F0BD2B
:1012C0007047012001F08ABA084810B50178084A31
:1012D000515C19B1001D01F01FF802E00C3000F064
:1012E0002DFFBDE81040002001F078BA400000203A
:1012F0000C00002008B5034A00924023024AFFF781
:101300007BFF08BD99260000800100200A4A0129C0
:1013100002EBC00007D0022907D0032907D0042917
:1013200007D00020704702207047042070470079E2
:1013300070474079704700002833000010B5FFF770
:10134000C0FF04210348FFF72FFF02490120487224
:1013500010BD0000540000202DE9F0478CB0FFF7CD
:1013600019FB18B100200CB0BDE8F087784C0020C4
:10137000C4F81804BFF34F8F60680290A5684FF05F
:101380000008284004EB800008E0216802988142B0
:1013900001D86160E6E7284004EB80000C3002A928
:1013A000FFF7A0FB0028F0D103AB029901EA050288
:1013B00004EB8202491CD26843F82020401C0291B1
:1013C0000228F2D3039800F00300022802D001287B
:1013D0004ED0A5E003985022810D8946B2EB905F74
:1013E00000D850210E4666F39F50039008315948AB
:1013F00000F0E3F9070078D000F028FA434608220D
:1014000003A9384600F03DFA029908F1080A29407C
:10141000681A8000001D864223D94D4D0C3530B12D
:10142000C2B204EB8101301A90460C3104E0294627
:10143000F2B2002590462846C6B25346384600F020
:1014400020FA0AEB08032DB1324629464FEA07007D
:1014500000F017FA029909F1030001EB90000290E5
:101460003AE004EB81015346324638460C31EFE74F
:101470000398C0F38311062900D3062161F3891074
:101480000390C0F38310801C8100324800F095F96E
:10149000070045D000F0DAF94346082203A9384690
:1014A00000F0EFF908F1080800260FE00298434623
:1014B00000EA0501401C04EB810102900422384639
:1014C0000C3100F0DEF908F10408761C0398C0F333
:1014D0008310B042EAD847B1D4F81054D4F81804B5
:1014E00068B1384600F0B8F92CE019E0687A0128B4
:1014F00004D12A6828463946126890476D68002D45
:10150000F4D1384600F0A8F90020FFF762F9D4F8CA
:10151000180408B9029860600020FFF75CF911E038
:10152000D4F8104404E0216820468968884764683C
:10153000002CF8D108480221008801EB004007A1E7
:1015400000F016F8FFF726FA80F001000BE7000024
:101550008002002068330000D00000204261636BED
:10156000656E647320666C757368656400000000C6
:1015700000231A4601F0B0B808B5012300926A466C
:1015800001F0AAF808BD1CB5CDE9002302236A4684
:1015900001F0A2F81CBD3EB5069C8DE81C0003239B
:1015A0006A4601F099F83EBD2DE9F0470E468046A7
:1015B0001C46924608293ED894F80C9000202073CF
:1015C0001946104600F01EFF0025B54206D218F855
:1015D00005201AA12046FFF747FC03E019A1204689
:1015E000FFF742FC6D1C082DEFD317A12046FFF733
:1015F0003BFC0025B54210D218F80570FEF78EFEB0
:101600000068C05D10F03E0F01D03A4600E02E2287
:101610000EA12046FFF728FC03E00DA12046FFF7AE
:1016200023FC6D1C082DE5D301222146504600F015
:10163000CBFE84F80C90BDE8F08700002025303206
:1016400078000000202020007C00000025630000BE
:1016500020000000104810B5FF21816000210160CA
:101660004160C0F81814C0F8141480F820140B4816
:1016700000F0F0F800280DD109480A490A4B401A39
:10168000C108002003E000BF23F82000401C88426E
:10169000FAD3002010BD0000800200206833000053
:1016A0006833000028330000B400002002480349DA
:1016B000401AC0087047000068330000283300005B
:1016C00013B56846FFF70AFB08B100201CBD0248AD
:1016D000009950F831001CBD2833000070B508484F
:1016E0000125D0F8104480F8205405E06572216887
:1016F0002046496888476468002CF7D170BD000017
:10170000800200202DE9FF4781460C9D00200C46F9
:101710002F7B2873984616462946184600F072FE1D
:10172000072E42D2DFE806F004090F161F2A360002
:1017300049462846FFF798FB37E049462846226885
:10174000FFF792FB31E0D4E9002349462846FFF732
:101750008BFB2AE0A0680090D4E900234946284684
:10176000FFF782FB21E0D4E90201CDE90001D4E9D1
:10177000002349462846FFF777FB16E004F10800EE
:1017800007C88DE80700D4E9002349462846FFF73B
:101790006BFB0AE004F108000FC88DE80F00D4E9E4
:1017A000002349462846FFF75FFB002229464046B2
:1017B00000F00AFE2F73BDE8FF872DE9F041858A0E
:1017C00080462D1F4819C01CB0FBF5F0C6B240463C
:1017D000FFF7BEFA041E19D00020207101206071AD
:1017E000E58000272546761EC4F800800BE04046C1
:1017F000FFF7AEFA60B16179491C61712860054656
:101800007F1CC0F80080B742F1D32046BDE8F081CC
:10181000204600F002F80020F8E72DE9F041457974
:1018200001466B1E002201E00968521C9A42FBD35C
:101830000F680146002605E038460C68FFF7A7FA56
:101840002146761CAE42F7D3BDE8F0810121001D90
:10185000FFF762BAFFF7B0BA10B504460121001DC8
:10186000FFF770FA10F0FF0F04D12046BDE81040DA
:10187000FFF7D3BF10BD38B501240094FFF7F2F98C
:1018800038BD38B500240094FFF7ECF938BD0000EE
:10189000064910B500204870091D0860BFF35F8F2E
:1018A0000349044800F046F8002010BD3400002031
:1018B000AC2C00007401002010B50020FEF789FF59
:1018C000F1EE100A20F09F00E1EE100ABFF35F8FE7
:1018D00005494020C1F880020020FEF77CFF20BFB0
:1018E00040BF20BF10BD000004E000E0024A1060CD
:1018F000101D0160704700002C7600400301034872
:101900001844C0F81425C0F8101570470070004046
:1019100002494058002800D0012070470070004064
:10192000034908B50844002202600068009008BD21
:1019300000700040016009684160AFF3008010B59D
:10194000D0E900215368994201D1002104E0D1E996
:101950000034A34202D01946816010BD08314160B5
:10196000F0E700000C4A10B502F58C730EE0991AEE
:10197000C91001EBD171491002EBC1010C6884421E
:1019800001D90B4602E005D201F108029A42EED3DA
:10199000002010BD486810BDCC2C000000B5FFF73A
:1019A000E1FF002800D1014800BD0000B82C000074
:1019B00008B5002242504058009008BD4058002809
:1019C00000D00120704708B50022425040580090D6
:1019D00008BDD0F80403084000D0012070474058EB
:1019E000002800D00120704708B50022425040581E
:1019F000009008BD0121B1EB507F01D1012070475B
:101A0000002070472DE9F05F0427204EDFF880901A
:101A1000834600244FF0030A4FF001080020FEF730
:101A2000D8FE08FA04F5354203D02046FFF780F8C7
:101A3000B8B10020FEF7CFFEFFB104F10104AE43C0
:101A4000E4B2EBD13846FFF7A9FFB9F8001003461E
:101A50000AEB01400F4A10A1FFF795FD3846BDE89B
:101A6000F09F154908FA04F000274A6810434860BF
:101A70008BF800403846FEF7AEFEB9F8001022465B
:101A80000AEB01400DA1FFF777FDDBE7FFFF0F0039
:101A9000D0000020492B000046756E6374696F6E9C
:101AA0003A2025732C206572726F7220636F646513
:101AB0003A2025732E00000020000020416C6C6F3E
:101AC0006361746564206368616E6E656C3A20259D
:101AD000642E00002DE9F84314460D0081462CD0F9
:101AE000002C2AD00026FFF72FF8174F4FF00308DD
:101AF000002824D04846FFF71BF8002821D01348BF
:101B000000EBC900C0F81055C0F81445009439889E
:101B10002B4608EB01404A460DA1FFF73CFD30463D
:101B2000FFF73CFF3988034608EB0140184A19A12A
:101B3000FFF729FD3046BDE8F8830E20FBE70726B6
:101B4000EDE70826EBE70000D000002000F00140A0
:101B500041737369676E6564206368616E6E656C5E
:101B60003A2025642C206576656E7420656E6420AD
:101B7000706F696E743A2025782C207461736B2025
:101B8000656E6420706F696E743A2025782E0000AF
:101B9000762B000046756E6374696F6E3A2025736C
:101BA0002C206572726F7220636F64653A20257312
:101BB0002E00000070B5044601260025A640FEF761
:101BC000C3FF18B12046FEF7B3FF80B10948066095
:101BD0002846FFF7E3FE034607480321074A00882B
:101BE00001EB004006A1FFF7CEFC284670BD08259A
:101BF000EEE7000004F50140D0000020AB2B000010
:101C000046756E6374696F6E3A2025732C20657279
:101C1000726F7220636F64653A2025732E00000096
:101C200070B50D4600F03AFC04000FD00020FEF71E
:101C3000D0FD207920B10020FEF7CDFD112070BD30
:101C40000120256020710020FEF7C5FD002070BD39
:101C500010B500F023FC002802D0002101600171C2
:101C600010BD00002DE9F041254C064612200D461E
:101C7000C4F808032348017C022918D0027C0146DD
:101C80004FF4807891F82E10012A12D00222C4F865
:101C9000042301270774466005810022C26021B336
:101CA000458390F82D103046FFF720FE25E01220E6
:101CB00002E0C2682AB10220C4F804031120BDE882
:101CC000F081C660058361B947463846FFF720FEBC
:101CD0000028FAD03846FFF723FE29463046FFF7A2
:101CE00005FE0220C4F8040307E029463046FFF74A
:101CF000FDFD4046FFF714FE27600020DFE70000EF
:101D000000700040E800002070B50C4623490546ED
:101D1000087C08B1112070BD01EB4500027F1AB9A3
:101D200011F82D2F521C0A70E1790177217A417741
:101D300021786278302301F0030103EA0212114393
:101D4000A2784FF4E06303EA02221143E2784FF4F1
:101D5000805303EA0232114322794FF4E02303EA6D
:101D60000242114362794FF4801303EA0252114395
:101D7000A2791B0103EA0262094B2846114303EBD7
:101D80000012C2F81815227AE179FFF7B7FD227A1E
:101D9000E1792846FFF7B2FD002070BDE800002081
:101DA000007000402DE9F0411E4C054694F82C00CF
:101DB00010B10820BDE8F08144F8101B1A492878BA
:101DC0000860091D68780860E878A0770127277700
:101DD0000020207060776060144EE0776FF0004064
:101DE000C6F808034FF48270FFF79AFDB015FFF7AD
:101DF00097FDA8780E49400181F800048020C91F92
:101E0000C1F88002C1F800010220C6F80403A07FD7
:101E100010B10120C6F804030348F0380760002021
:101E2000C8E70000E8000020F075004000700040A6
:101E300007E000E0044890F82E0008B1002000E020
:101E40000420024908447047E80000200070004068
:101E50002DE9F04106460D464FF4803400681746E0
:101E6000AC404BB14FF4A07101EB8501FFF7A0FD31
:101E70003068C0F8044301E0C0F80843306800EB64
:101E80008500C0F84075BDE8F081000001680122BE
:101E90000A600079034A00EB400002EB8000022157
:101EA0000172704718010020F0B40468049E40F2EB
:101EB0000115D4F800728D40AF43C4F80072046875
:101EC000D4F800521D43C4F800523346F0BCFFF76B
:101ED000BFBF00002DE9F04104460E4600792C49B1
:101EE00000EB400001EB8007387A10B10820BDE814
:101EF000F0813A60706800254FF4A078786006E0C1
:101F000008EB85012068FFF753FD6D1CEDB2607989
:101F1000A842F5D82068F178000B40B200284FEABB
:101F2000411106DA00F00F0000F1E02080F8141DE6
:101F300003E000F1E02080F8001420680122000B8B
:101F400040B200F01F0302FA03F14009800000F1E3
:101F5000E020C0F88012C0F8001120687178D0F835
:101F6000043561F30103C0F804352068B178D0F876
:101F7000083561F30103C0F8083520683178D0F8DE
:101F8000103561F30303C0F810353A720020AEE754
:101F9000180100200149024800F048BC240100203B
:101FA000002000402DE9F0410546007916460F4615
:101FB00000EB40012D4A01EBC00102EB810494F8D3
:101FC0002A1011B10820BDE8F081294951F82010EC
:101FD0002868FFF725FE08B11120F4E739462846A6
:101FE000FEF70EFC66603869206030004FF0010695
:101FF0002FD03F7F4FF48E712868FFF7E4FC4FF439
:10200000A2712868FFF7DFFC28681A49C0F804139A
:1020100028684FEA4711000B40B2002806DA00F0AA
:102020000F0000F1E02080F8141D03E000F1E02033
:1020300080F800142868000B40B200F01F0206FA76
:1020400002F14009800000F1E020C0F88012C0F8E1
:10205000001128680421C0F800150020A061E0618B
:1020600084F8290044F8140FA675ACE72401002079
:102070007C2C0000800002002DE9F0470546007925
:102080000B4600EB400101EBC000234901EB80044B
:10209000284600F043F810B11120BDE8F0874FF05A
:1020A0000008C4F82080A360626184F828804FF49F
:1020B0008E76474631462868FFF785FC28684FF042
:1020C0000109C0F808902146286800F04CFB6068C0
:1020D00000BBD5F800A00EE094F8280008B10F2747
:1020E00016E031465046FFF769FC0028F4D021463F
:1020F000504600F038FB216A60698142F1D33146D5
:102100002868FFF75BFC0028F9D02868C0F80C901D
:10211000C4F814803846C0E724010020007900EBA1
:10212000400101EBC000044901EB80004069002838
:1021300000D0012070470000240100202DE9F04765
:10214000044600794FF0000900EB400101EBC000AC
:10215000254901EB80072068C0F80095786880B1B8
:1021600020682249C0F8081320680121000B40B202
:1021700000F01F0291404009800000F1E020C0F80B
:1021800080112068D0F80C25D0F81485D0F80865A7
:10219000D0F810554FF0FF31C0F81415C0F80C15E9
:1021A0002068C0F80815C0F81015501C02D0104661
:1021B000FEF792FFB8F1FF3F02D04046FEF78CFFDA
:1021C000681C02D02846FEF787FF701C02D03046FC
:1021D000FEF782FF2068FFF73BFD87F82A90C7F8DB
:1021E0000490BDE8F0870000240100208402020072
:1021F0000149024800F0C6BB500100200020004009
:102200002DE9F0410546164600790F46154A00EBC8
:10221000C00102EB810494F8201011B10820BDE840
:10222000F081114951F820102868FFF7F9FC08B136
:102230001120F4E739462846FEF71DFB6660386931
:1022400020601EB1397F2846FEF70CFC2868082163
:10225000C0F800150020A061E0610121606184F8F0
:102260002010DCE750010020802C00002DE9F04711
:1022700004460E460079204900EBC00001EB8005C2
:1022800017463046FFF7B6FB30B1204600F036F86F
:1022900020B11120BDE8F0871020FBE76F61AE6030
:1022A0004FF49076002731462068FFF79DFB4FF4EE
:1022B000AC7841462068FFF797FB2068AA686969F7
:1022C000C0F84425C0F8481520680121816068687D
:1022D00078B9B14649462068FFF781FB064641467A
:1022E0002068FFF77CFB0643F4D000B10F270020E5
:1022F00068613846CEE700005001002000790549AA
:1023000000EBC00001EB80004069002800D00120F4
:1023100070470000500100202DE9F0470446007985
:10232000274900EBC00001EB800720684FF000094F
:10233000C0F80095786880B120682249C0F8081379
:1023400020680121000B40B200F01F0291404009BB
:10235000800000F1E020C0F880112068D0F80C2542
:10236000D0F81485D0F80865D0F810554FF0FF313B
:10237000C0F80C15C0F814152068C0F80815C0F88E
:102380001015501C02D01046FEF7AFFEB8F1FF3F0B
:1023900002D04046FEF7A9FE681C02D02846FEF790
:1023A000A4FE701C02D03046FEF79FFE2068FFF7A7
:1023B0004FFC87F82090C7F80490BDE8F087000034
:1023C000500100201003020010B50C46017A0529C7
:1023D00008D0407A38B1084808A102682046FEF7C4
:1023E00043FD00E01AB106A12046FEF73DFD204660
:1023F000BDE81040FEF745BD8C00002025730000AD
:102400000D0A000038B5C3880D46044633B114A048
:10241000009015A216A12846FEF726FD217A05296F
:102420001CD0607A48B1A088FEF770FF164951F8B9
:10243000202016A12846FEF717FDA0880021FFF7EF
:102440003FF903461049207A143951F8202001B091
:102450002846BDE830400EA1FEF706BD38BD00009D
:102460001B5B306D000000001B5B313B33316D00A6
:1024700025734C6F67732064726F707065642028D9
:1024800025642925730D0A008C00002025730000A7
:102490003C25733E2025733A200000000349884202
:1024A00001D1034870470020704700000020004021
:1024B0002800002070B5054688690C4600284FF4B6
:1024C000847128460AD0FFF77EFAD5F81805626AAB
:1024D000E1688854606A401C606270BDFFF773FA5F
:1024E000D5F8180570BD1FB501238DF80030CDE972
:1024F0000121D0E90012684690471FBD1FB5012396
:102500008DF800308DF808100192D0E9001268466D
:1025100090471FBD2DE9F04105460078002824D1E1
:1025200005216868FFF79EFB08B1FEF747F9104FD9
:10253000DFF84080032638880FA106EB0040D8F86A
:102540000420FFF719F80024686811A130F914205D
:10255000388806EB0040FFF70FF8641C052CF3DB0E
:10256000D8F80410491CC8F80410BDE8F081000038
:10257000D000002000000020414443206576656EB5
:1025800074206E756D6265723A202564000000004B
:10259000256400000EB5124A07CA8DE807001048EE
:1025A00010491438FFF7FEFB08B1FEF707F969463A
:1025B0000020FFF7A9FB08B1FEF700F905210A4842
:1025C000FFF750FB08B1FEF7F9F8074805210A307C
:1025D000FFF748FB002801D0FEF7F0F80EBD000021
:1025E000402B000015250000D4000020054810B540
:1025F0000078FFF7DFFA002803D0BDE81040FEF7AF
:10260000DDB810BD000000203EB5FEF7EDFB08B1BF
:10261000FEF7D4F81C491D4AD1E90301CDE90101B7
:1026200003208DF80600184801A9001DFFF752FC91
:1026300008B1FEF7C3F8144C241D2068D0F810052B
:10264000134A0123C2400020014600902046FFF7B4
:102650002BFC2046FFF71AFC246804F5A074FFF752
:10266000E9FB05460B48FFF7CDF908B1FEF7A6F8E0
:1026700008482A4621460078FFF72CFA002801D0A6
:10268000FEF79CF83EBD00002C2B000065270000E3
:1026900000A861000000002070B50D4C0020D2B2EF
:1026A0002070201D0B4D0378EB5C1BB1001DFFF764
:1026B000DDFD02E00C30FFF7DFFC08B1FEF77EF82D
:1026C0006078002802D021780029FAD070BD00007F
:1026D0003C0000200C0000202DE9F84F204D9246D0
:1026E000894606469846012269461846AF68FEF7B5
:1026F000FDF858B3009800210446801C09E000BF93
:1027000000EA07035AF8212005EB8303401C491C0B
:10271000DA604145F4D34FEA164AFEF745F94AEA32
:102720000041601C384005EB80003C4005EB840212
:10273000C160D06866F3C50068F3891069F39F2013
:1027400020F00300401C20F00400D06095F8200425
:1027500002E000BFFEF700FE0028FBD1BDE8F88FC5
:1027600080020020704770B50C4605464FF48E710C
:10277000FFF729F9216AA068415C206A401C2062A9
:10278000C5F81C1570BD1FB500228DF80020029100
:10279000816801914261D0E90012684690471FBDEF
:1027A0001FB50A4601788DF8001041680191017A41
:1027B0008DF80810C0680390044850F822100838BB
:1027C00050F82220684690471FBD000018000020E6
:1027D00001490120087070473C00002010B588B006
:1027E000044620220E496846FDF79CFD0620009015
:1027F000C01F0190029003904FF0EB7006900CB157
:10280000084A00E0002269460748FEF7F9FA08B1D5
:10281000FDF7D4FF0448001F447008B010BD00004D
:10282000F02D0000D1270000400000202DE9FF47D7
:102830000C4605464FF40071FFF7CBF801274FF423
:102840000178002618B34FF4927949462846FFF7DD
:10285000B5F8E0B149462846FFF7B5F8C5F8088352
:1028600094F8290000B96F6002208DF80000D5F8B7
:102870008004C5F880040390A0690290E06801908C
:10288000A661E661D4E900126846904728E0042179
:102890002846FFF79EF818B34FF484712846FFF7D7
:1028A0008DF8E8B121462846FFF704FE616AA06969
:1028B000884215D1E06938B1E268616AA061206997
:1028C000E6616662E06008E094F8290000B96F6094
:1028D000C5F80883A661E268616A2046FFF703FE37
:1028E0004FF48E7841462846FFF768F878B1206AA1
:1028F0006169884202D294F8280020B341462846F4
:10290000FFF761F8616911B12046FFF73CFF4FF412
:10291000A27841462846FFF751F8002818D04146D2
:102920002846FFF750F894F8290000B12F60A069FD
:1029300000280DD0A661E268616A04B02046BDE8B7
:10294000F047FFF7D0BD21462846FFF70CFFDEE732
:10295000BDE8FF871FB50A4601788DF80010416871
:102960000191017A8DF80810C0680390044850F86E
:102970002210083850F82220684690471FBD0000FA
:10298000180000202DE9FF410C464FF492770546D0
:102990003946FFF724F80026C0B139462846FFF72C
:1029A00023F802208DF80000D5F88004C5F88004D3
:1029B0000390D5F83C058DF80800E0680190A66109
:1029C000E661D4E900126846904723E04FF4887727
:1029D00039462846FFF703F8E0B139462846FFF7A5
:1029E00003F8D5F83C15A069884213D1E06960B1BD
:1029F000E268D5F8000220F02000C5F80002E06986
:102A0000A0612069E661E06001E0A661E26820461D
:102A1000FFF774FD4FF4A27739462846FEF7DFFF33
:102A200060B139462846FEF7DFFFA06930B1A661E4
:102A3000D5F83C152046E268FFF760FD4FF490772B
:102A400039462846FEF7CBFF002813D039462846E2
:102A5000FEF7CAFF606900280CD0D5F84C058DF848
:102A600000608DF80800A06801906661D4E900124A
:102A700068469047BDE8FF812DE9F05F8346DDE9B8
:102A80000A4A994690460D460846012703E000BFD2
:102A9000B0FBF8F07F1C4045FAD2B94500D94F464B
:102AA0005FEACA7012D18CB15FEA8A7002D5B9F1BF
:102AB000000F01D0202607E0302605E031465846B9
:102AC000641EFDF757FF0CB1A742F7D35FF0010674
:102AD000B9F1010F02D9A9F1010903E0B5FBF6F044
:102AE000404502D306FB08F6F2E7DFF83C9000BF52
:102AF000B5FBF6F000FB165519F800105846FDF727
:102B000039FFB6FBF8F6002EF2D15FEACA7009D0A1
:102B1000002C07D0A74205D220215846641EFDF79D
:102B200029FFF5E7BDE8F09F842C000001000700B5
:102B300000800040000400000000000700000000CA
:102B40000000000002000001006E7266785F707085
:102B5000695F6368616E6E656C5F616C6C6F63006A
:102B60006E7266785F7070695F6368616E6E656CC7
:102B70005F66726565006E7266785F7070695F632C
:102B800068616E6E656C5F61737369676E006E720B
:102B900066785F7070695F6368616E6E656C5F66B2
:102BA0006F726B5F61737369676E006E7266785FD8
:102BB0007070695F6368616E6E656C5F656E61629F
:102BC0006C65006E7266785F7070695F6368616ED5
:102BD0006E656C5F64697361626C65006E726678C5
:102BE0005F7070695F67726F75705F616C6C6F6347
:102BF000006E7266785F7070695F67726F75705F84
:102C000066726565006E7266785F7070695F677284
:102C10006F75705F656E61626C65006E7266785F7D
:102C20007070695F67726F75705F64697361626C01
:102C300065006E7266785F7070695F6368616E6E62
:102C4000656C735F72656D6F76655F66726F6D5FE1
:102C500067726F7570006E7266785F7070695F631F
:102C600068616E6E656C735F696E636C7564655FD9
:102C7000696E5F67726F757000000000951F00003D
:102C8000F1210000303132333435363738394142A2
:102C90004344454600000000000000000000000022
:102CA000000000000000000000000000942C000064
:102CB000AC2C000004000000556E6B6E6F776E2028
:102CC0006572726F7220636F64650000000000001F
:102CD000FC31000001000000BC30000002000000D8
:102CE000B02E00000300000030310000040000009E
:102CF0008431000005000000643000000600000080
:102D000000300000070000006C31000008000000E7
:102D10007830000009000000DC3000000A000000EC
:102D2000E43100000B000000982E00000C000000B1
:102D3000903000000D000000343200000E00000052
:102D40005C3100000F00000098310000100000000E
:102D5000CC3100001100000048320000800000006B
:102D60001830000081000000542F00008200000095
:102D7000142F000083000000F42E000084000000E7
:102D8000302F0000850000003C300000860000006D
:102D90004431000090000000E02F0000910000008E
:102DA000D42E000092000000A43000000082000039
:102DB000AC31000001820000F83000000282000007
:102DC0001431000000840000702F00000184000016
:102DD0000832000002840000B82F000003840000C5
:102DE000942F0000F5120000C9120000C11200006B
:102DF000FFFFFFFFFFFFFFFFFFFFFFFFFFFFFFFFE3
:102E000000000000000000000000D60107010000E3
:102E100000404040404040404040414141414140ED
:102E200040404040404040404040404040404040A2
:102E30004005020202020202020202020202020231
:102E40000220202020202020202020020202020236
:102E5000020290909090909010101010101010108E
:102E6000101010101010101010101010020202029A
:102E700002028888888888880808080808080808DE
:102E800008080808080808080808080802020202DA
:102E900040000000112E00004E52465F4552524F36
:102EA000525F494E56414C49445F444154410000F1
:102EB0004E52465F4552524F525F534F465444451F
:102EC000564943455F4E4F545F454E41424C454441
:102ED000000000004E52465F4552524F525F464539
:102EE00041545552455F4E4F545F454E41424C450B
:102EF000440000004E52465F4552524F525F4D55BE
:102F00005445585F554E4C4F434B5F4641494C45E5
:102F1000440000004E52465F4552524F525F4D559D
:102F20005445585F4C4F434B5F4641494C45440024
:102F30004E52465F4552524F525F4D555445585F71
:102F4000434F4E445F494E49545F4641494C4544C6
:102F5000000000004E52465F4552524F525F4D55A1
:102F60005445585F494E49545F4641494C454400D9
:102F70004E52465F4552524F525F424C455F495058
:102F800053505F52585F504B545F5452554E43411B
:102F9000544544004E52465F4552524F525F424C98
:102FA000455F495053505F504545525F52454A4531
:102FB00043544544000000004E52465F4552524F74
:102FC000525F424C455F495053505F4C494E4B5FF6
:102FD000444953434F4E4E4543544544000000007E
:102FE0004E52465F4552524F525F4150495F4E4FDD
:102FF000545F494D504C454D454E544544000000EA
:103000004E52465F4552524F525F4E4F545F53559A
:1030100050504F52544544004E52465F4552524F15
:10302000525F4D4F44554C455F4E4F545F494E499A
:103030005449414C495A4544000000004E52465FF5
:103040004552524F525F4D4F44554C455F414C5293
:10305000454144595F494E495449414C495A4544B8
:10306000000000004E52465F4552524F525F4E4F95
:10307000545F464F554E44004E52465F4552524FA4
:10308000525F494E56414C49445F535441544500A8
:103090004E52465F4552524F525F444154415F5336
:1030A000495A45004E52465F4552524F525F494F72
:1030B0005F50454E44494E47000000004E52465F67
:1030C0004552524F525F5356435F48414E444C4520
:1030D000525F4D495353494E470000004E52465FE0
:1030E0004552524F525F494E56414C49445F4C4500
:1030F0004E475448000000004E52465F4552524F22
:10310000525F4452565F5457495F4552525F414E99
:1031100041434B004E52465F4552524F525F44521C
:10312000565F5457495F4552525F444E41434B00EE
:103130004E52465F4552524F525F494E5445524E91
:10314000414C00004E52465F4552524F525F53541D
:103150004F524147455F46554C4C00004E52465F2A
:103160004552524F525F4E554C4C00004E52465FF6
:103170004552524F525F494E56414C49445F50416F
:1031800052414D004E52465F4552524F525F4E4F94
:103190005F4D454D000000004E52465F4552524F74
:1031A000525F464F5242494444454E004E52465F9C
:1031B0004552524F525F4452565F5457495F4552F1
:1031C000525F4F56455252554E0000004E52465FD8
:1031D0004552524F525F494E56414C49445F41441B
:1031E000445200004E52465F4552524F525F494E84
:1031F00056414C49445F464C414753004E52465F4E
:1032000053554343455353004E52465F4552524F28
:10321000525F424C455F495053505F4348414E4EC8
:10322000454C5F414C52454144595F4558495354C0
:10323000530000004E52465F4552524F525F544970
:103240004D454F55540000004E52465F4552524F77
:10325000525F4255535900007761726E696E670084
:1032600064656275670000001B5B313B33306D00A5
:103270001B5B306D000000001B5B313B33316D0088
:103280001B5B313B33326D001B5B313B33336D00D5
:103290001B5B313B33346D001B5B313B33356D00C1
:1032A0001B5B313B33366D001B5B313B33376D00AD
:1032B000696E666F000000006572726F7200000038
:1032C00050525300534141444300000054494D457E
:1032D0005200000055415254000000005541525424
:1032E000450000007077725F6D676D74000000002C
:1032F00062616C6C6F632E6C6F675F6D656D706F74
:103300006F6C0000617070008033000000000020CE
:10331000D40000002007000054340000D400002036
:10332000D425000030070000C0320000000000007B
:10333000C432000000000000CC3200000000000099
:10334000D432000000000000DC3200000000000069
:10335000E432000000000000F03200000000000332
:103360000433000000000303680000206000002018
:1033700068000020C0010020CC00002018000000E0
:10338000000000000000000000000000000000003D
:10339000000000000000000000000000000000002D
:1033A000000000000000000000000000000000001D
:1033B000000000000000000000000000000000000D
:1033C000000000000020004000000000002000403D
:1033D00000000000E42D00000000000000000000DC
:1033E00000000000000000000000000000000000DD
:1033F000000000000000000000000000B8320000E3
:1034000058320000B032000060320000703200001C
:1034100068320000783200008032000088320000FC
:103420009032000098320000A0320000A832000064
:103430000090D00300000000000000000000000029
:10344000000000000000000000000000000000007C
:043450000000000078
:0400000500000201F4
:00000001FF
